:10000000A42A82004F347C2957345B345F345D343A
:1000100072297C294D345134553459347B34FF34A2
:100020007C297C2906293F347C290229DF34FD34D0
:100030007C297C297C299D34BD34BF34DD34FB34DC
:100040007C297C2999349B34BB34DB34F734F93474
:100050007C297C297F349734B934D734D934F534AA
:100060007C297C2993349534B534B734D534F334B2
:100070007C297C297C299134B334D334F134EF3496
:100080007C297C298F34B134D134CF34EB34ED3436
:100090007C297C298D348B34AF34AD34CD34E934B4
:1000A0007C297C297C29AB347C29CB34E7347C291E
:1000B0007C2967293D347734C9347C29A9347C29CB
:1000C0007C297C299F347C297C297C297C297D34CE
:1000D0007C297C29C5347C29A53485347C297C295C
:1000E0007C29E1348734C334A334A1348334753498
:1000F0005F297C294334C1346B34453481347529FC
:100100007C297C297C297C29533423297C297C293E
:100110007C297C297C297C297C297C297C297C29B7
:100120007C297C2909297C297C2900297C297C2996
:100130007C297C297C297C297C297C297C297C2997
:100140000C297C297C297C297C297C297C297C29F7
:1001500012297C297C297C297C297C297C297C29E1
:1001600018297C297C297C297C297C297C297C29CB
:100170007C297C297C297C297C297C297C297C2957
:100180007C297C297C297C297C297C297C297C2947
:100190007C297C297C2947347C297C297C297C2961
:1001A0007C297C297C297C297C297C297C297C2927
:1001B0007C297C297C2979347C297C297C297C290F
:1001C0007C297C297C297C297C297C297C297C2907
:1001D0007C297C2937297C2961342D297C297C299B
:1001E00063347929733465347C29633467347C291A
:1001F0007C297C297C2941297C2923294B297C299C
:100200009E1F7C291A141A1A1A1039349E1E0E29A0
:1002100037349E1E142935349E1E37349A141A1A08
:100220009A1033349E1E35341A151A1A1A113134A5
:100230009D1C7C291A1E00343330B6219130EB21ED
:100240003230B62100341D1F7C291A1E0034313093
:10025000B621CD30EB21303021291D1D7C291A1EFD
:1002600000343D30B6216130EB213C3021299D1D09
:100270007C291A1E00343D30B6216330EB213C301E
:1002800021299D1E7C291A1E00343D30B62165307F
:10029000EB213C3021291D1E7C291A1E00343D30E3
:1002A000B6216730EB213C3021291E1C7C291A1E07
:1002B00000343930B6219930EB21383021291E1E07
:1002C0004B341A1E003402309B06972100349E1DC9
:1002D0007C291A1E003404309B0697213B301B1DDD
:1002E000FE3921291E197C2941349E187C299A1235
:1002F00000349D1F7C29413494092E30B6211E30D4
:1003000091001A1A11119A1991109A1E911111083F
:10031000B62114089100910D11081E39B621940ED2
:10032000940D14081E39212901301B069B00ED3065
:10033000F2212B220508F8391B0485001B08F22145
:100340002B2AA3210030962125309100AA21910B60
:10035000A6290800FF3092006400920BAD29080026
:1003600090000F020319080010088F0090000A3057
:10037000A52108309100A300901B8515901F8511C1
:100380000A30AB2105120A30AB2105160A30AB2129
:10039000900D910BBC298316851583129101920152
:1003A000851DDA296400910BD029920BD0291A1BE4
:1003B0000800E6291A1B080091018519E129910B13
:1003C000DD2985158316851183120800E121910A24
:1003D000A30BC02908009700B6211708FE39B621E3
:1003E0001708080094009501861400000610831673
:1003F00086100000061083120830910083168614C0
:1004000083128618012A14180614141C0610940C62
:100410000318950A861C0A2A910B012A86180E2AAF
:1004200015180610151C0614861C142A8618162A80
:100430000614861C192A83160614831286181E2A8F
:10044000861C202A0830AB21861083168610831262
:100450001430AB21080096011A169A1186148316DF
:1004600086148312861C3D2A6400061B322A9A1EBB
:10047000322AA11FE02BA1138C2A861C3D2A0830AA
:1004800091008618412A940C06189417061C9413A0
:10049000861C482A910B412A86184C2A861C4E2A13
:1004A0008618502A861C522A88221430AB2116083E
:1004B00003195C2A96032E2AE130140203197B2AC1
:1004C000E030140203197F2AF03014020319812A44
:1004D0009A1D732A1230140203192B2A5930140260
:1004E00003192B2A080083301402031D08009A15F3
:1004F0000330940008005521073096002C2A9A15E5
:100500002E2A1A122E2A86148316861483120800A5
:10051000861083168610862A0F30B6211A170F30E0
:10052000B6211630930085199C2A910B932A920BC1
:10053000932A9421930B932A051283160611831292
:10054000FF30A521A11FD22B1D2307309A008F0158
:10055000103039239D003A239E003A239F003A230E
:10056000A0003A23A100061CB32AFF30F221073075
:10057000A121F3309F21FF309F211E1BC12AA11F03
:10058000D22B0230B6210230B6211D189A161A0855
:10059000073903198C2A9A1EEC2A2B221A19DD2AF4
:1005A0001E1BD72AC7239A1BD72AA1138C2A9A1855
:1005B000DD2A073014020319422B941FE12A7C2103
:1005C000C72A140A9A19803E0120003E0319C72A3F
:1005D0001A1EFE39B021C72A06129C01A201910100
:1005E0004030920883226400861CFD2A910BF32A76
:1005F000920BF32A88229421192B7D23003E031DA0
:10060000192B3A2314020319A20A5A301402031DAB
:10061000152B22081C02031DEC2AFF3094007C21BC
:100620001B1097219A160616C72A10301C020319B0
:10063000EC2A1C0894007C21EF2A831218308500D4
:1006400018308600831681138501C7308600831217
:10065000080088001C0889009C0A8316081555307C
:100660008900AA3089008814081E342B880183125F
:1006700008009C001C0889009C0A83160814831239
:10068000080808001A123330EB213130EB214330D7
:10069000EB217D239923163014020319542B1E30AD
:1006A000140203196C2BA42A9C017D2366301402CA
:1006B0000319682B9923140829235A3014020319AB
:1006C000472B0F301C02031D552B5A3094005A2B18
:1006D0001C08031D9C03552B10309C007D239F2379
:1006E0009800980E99237D239F231804292399238A
:1006F00014301C02031D6E2B472B2B22941B922BB4
:100700001A1E922B9A19922B910159309523583029
:100710009523113095231230952314309523110819
:10072000031900349A1E01347D2B14020319910A17
:100730000800140A0120003E03190800EB2991016A
:1007400092011630BE231E30BE232630BE23253034
:10075000BE232E30BE233630BE233D30BE233E3076
:10076000BE234630BE231C30BE233230BE23213090
:10077000BE232330BE232430BE232B30910A140223
:100780000319C42B120808001108920008009A17D8
:100790001A08F7381F02031D080020081402031965
:1007A0009A130800A11314309C00210829238611F4
:1007B0008616E7232B221A1EDA2BC7239A1BDA2B65
:1007C000A11714309C0021082923E723A42AEA2337
:0807D000061FE72B8030A5296C
:084000000000010001000900AD
:02400E00F73F7A
:104200001C003A00430034001C005A00FF00FF006D
:10421000FF00FF00FF00FF00FF00FF00FF00FF00A6
:0A422000FF00FF00F7007600FF002A
:00000001FF
